
 KEYBOARD

 Start     Length     Name                   Class
 0001:0000 001F5H     _TEXT                  CODE
 0002:0000 00039H     _DATA                  DATA

 Origin   Group
 0002:0   DGROUP

 Address   Export                  Alias

 0001:006D ANSITOOEM               ANSITOOEM
 0001:00D5 ANSITOOEMBUFF           ANSITOOEMBUFF
 0001:0184 DISABLE                 DISABLE
 0001:016B ENABLE                  ENABLE
 0001:012C ENABLEKBSYSREQ          ENABLEKBSYSREQ
 0001:01DD GETBIOSKEYPROC          GETBIOSKEYPROC
 0001:00BB GETKBCODEPAGE           GETKBCODEPAGE
 0001:00A1 GETKEYBOARDTYPE         GETKEYBOARDTYPE
 0001:00C8 GETKEYNAMETEXT          GETKEYNAMETEXT
 0001:019B GETTABLESEG             GETTABLESEG
 0001:00F0 INQUIRE                 INQUIRE
 0001:00AE MAPVIRTUALKEY           MAPVIRTUALKEY
 0001:01B0 NEWTABLE                NEWTABLE
 0001:0087 OEMKEYSCAN              OEMKEYSCAN
 0001:007A OEMTOANSI               OEMTOANSI
 0001:00E2 OEMTOANSIBUFF           OEMTOANSIBUFF
 0001:0114 SCREENSWITCHENABLE      SCREENSWITCHENABLE
 0001:01C7 SETSPEED                SETSPEED
 0001:0060 TOASCII                 TOASCII
 0001:0094 VKKEYSCAN               VKKEYSCAN
 0001:0054 WEP                     WEP

  Address         Publics by Name

 0001:006D       ANSITOOEM
 0001:00D5       ANSITOOEMBUFF
 0002:0028       bios_proc
 0001:0184       DISABLE
 0001:016B       ENABLE
 0001:012C       ENABLEKBSYSREQ
 0002:0030       fSysReq
 0001:01DD       GETBIOSKEYPROC
 0001:00BB       GETKBCODEPAGE
 0001:00A1       GETKEYBOARDTYPE
 0001:00C8       GETKEYNAMETEXT
 0001:019B       GETTABLESEG
 0001:00F0       INQUIRE
 0002:0031       inquireData
 0002:0037       iqdNumFunc
 0001:002D       keybd_int
 0001:0000       KEYBOARD16
 0001:00AE       MAPVIRTUALKEY
 0001:01B0       NEWTABLE
 0002:002C       nmi_vector
 0001:0087       OEMKEYSCAN
 0001:007A       OEMTOANSI
 0001:00E2       OEMTOANSIBUFF
 0001:0114       SCREENSWITCHENABLE
 0001:01C7       SETSPEED
 0001:0060       TOASCII
 0001:0094       VKKEYSCAN
 0001:0054       WEP
 0000:0000  Imp  WOW16Call            (KERNEL.500)
 0000:0000  Abs  __acrtused
 0000:0000  Imp  __MOD_COMMDLG        (KERNEL.532)
 0000:0000  Imp  __MOD_DGDI           (KERNEL.525)
 0000:0000  Imp  __MOD_DKERNEL        (KERNEL.521)
 0000:0000  Imp  __MOD_DUSER          (KERNEL.523)
 0000:0000  Imp  __MOD_GDI            (KERNEL.524)
 0000:0000  Imp  __MOD_KERNEL         (KERNEL.520)
 0000:0000  Imp  __MOD_KEYBOARD       (KERNEL.526)
 0000:0000  Imp  __MOD_MMEDIA         (KERNEL.531)
 0000:0000  Imp  __MOD_SHELL          (KERNEL.528)
 0000:0000  Imp  __MOD_SOUND          (KERNEL.527)
 0000:0000  Imp  __MOD_TOOLHELP       (KERNEL.530)
 0000:0000  Imp  __MOD_USER           (KERNEL.522)
 0000:0000  Imp  __MOD_WINSOCK        (KERNEL.529)

  Address         Publics by Value

 0000:0000  Imp  WOW16Call            (KERNEL.500)
 0000:0000  Imp  __MOD_SHELL          (KERNEL.528)
 0000:0000  Imp  __MOD_MMEDIA         (KERNEL.531)
 0000:0000  Imp  __MOD_COMMDLG        (KERNEL.532)
 0000:0000  Imp  __MOD_USER           (KERNEL.522)
 0000:0000  Imp  __MOD_WINSOCK        (KERNEL.529)
 0000:0000  Imp  __MOD_TOOLHELP       (KERNEL.530)
 0000:0000  Imp  __MOD_DKERNEL        (KERNEL.521)
 0000:0000  Imp  __MOD_SOUND          (KERNEL.527)
 0000:0000  Imp  __MOD_GDI            (KERNEL.524)
 0000:0000  Imp  __MOD_KERNEL         (KERNEL.520)
 0000:0000  Imp  __MOD_KEYBOARD       (KERNEL.526)
 0000:0000  Imp  __MOD_DGDI           (KERNEL.525)
 0000:0000  Abs  __acrtused
 0000:0000  Imp  __MOD_DUSER          (KERNEL.523)
 0001:0000       KEYBOARD16
 0001:002D       keybd_int
 0001:0054       WEP
 0001:0060       TOASCII
 0001:006D       ANSITOOEM
 0001:007A       OEMTOANSI
 0001:0087       OEMKEYSCAN
 0001:0094       VKKEYSCAN
 0001:00A1       GETKEYBOARDTYPE
 0001:00AE       MAPVIRTUALKEY
 0001:00BB       GETKBCODEPAGE
 0001:00C8       GETKEYNAMETEXT
 0001:00D5       ANSITOOEMBUFF
 0001:00E2       OEMTOANSIBUFF
 0001:00F0       INQUIRE
 0001:0114       SCREENSWITCHENABLE
 0001:012C       ENABLEKBSYSREQ
 0001:016B       ENABLE
 0001:0184       DISABLE
 0001:019B       GETTABLESEG
 0001:01B0       NEWTABLE
 0001:01C7       SETSPEED
 0001:01DD       GETBIOSKEYPROC
 0002:0028       bios_proc
 0002:002C       nmi_vector
 0002:0030       fSysReq
 0002:0031       inquireData
 0002:0037       iqdNumFunc

Program entry point at 0001:0000
